:100000000C94EB040C9433050C9433050C943305D9
:100010000C9433050C9433050C9433050C94330580
:100020000C9433050C9433050C9433050C94501C3C
:100030000C9433050C94271C0C9433050C94330555
:100040000C9433050C9433050C9433050C94011C6B
:100050000C9433050C9433050C9433050C949B20BD
:100060000C9433050C9433050C9433050C94330530
:100070000C9433050631FF0974A10109751500269A
:10008000FF009520750881020976150026FF00956E
:100090002075089102C005010902A1010901A10012
:1000A0008501050919012908150025019508750123
:1000B00081020501093009311581257F95027508F6
:1000C000810609381581257F950175088106050C83
:1000D0000A38021581257F950175088106C0C00583
:1000E000010980A10185021601002637001A81004E
:1000F0002AB700751095018100C0050C0901A10106
:100100008503160100269C021A01002A9C02751024
:1001100095018100C005010906A101050719E02923
:10012000E715002501950875018102950175088183
:1001300001050819012905950575019102950175BB
:100140000391010507190029FF150026FF009506F8
:1001500075088100C0732530325820007225303474
:1001600058200073656E6420253032583A202530BF
:1001700032580A0073656E642039443A20253032C3
:10018000580A007225303258200073656E6420379B
:10019000303A20253032580A0073656E64203943A6
:1001A0003A20253032580A000A456E61626C65209B
:1001B00057696E6B65793A20000A496E6869626911
:1001C00074205265706561743A20005B4F4C445D49
:1001D000005B4E45575D000A4B6579626F61726442
:1001E00020547970653A200025583A253038622528
:1001F000730A000A202030313233343536370A0092
:10020000706339385F6C65643A20253032580A00D3
:100210007573625F6C65643A20253032580A004C71
:1002200045443A20253032580A000A4C6F6F70203E
:1002300073746172742E0A000A55534220636F6E04
:10024000666967757265642E0A000A544D4B3A63FD
:1002500031363865322F4C5546413A643661376441
:10026000660A0009025400030100A03209040000DC
:1002700001030101000921110100012240000705CD
:10028000810308000A090401000103010200092199
:1002900011010001227F0007058203080001090403
:1002A00002000103000000092111010001222200C7
:1002B000070583032000011201100100000008ED72
:1002C000FE01980101010200013003500043003992
:1002D00000380020006B006500790062006F00614B
:1002E0000072006400200063006F006E00760065FD
:1002F00000720074006500720000000E0374002E8E
:10030000006D002E006B002E000000040309047332
:10031000797374656D3A20253034580A00636F6E26
:1003200073756D65723A20253034580A003F004DD0
:100330003E2000433E20000A00257500363A207713
:100340006865656C5F74696D655F746F5F6D61781A
:100350003A20000A00257500353A20776865656CFB
:100360005F6D61785F73706565643A20000A0025EF
:100370007500343A2074696D655F746F5F6D6178E4
:100380003A20000A00257500333A206D61785F73CA
:10039000706565643A20000A00257500323A2069CC
:1003A0006E74657276616C286D73293A20000A00BC
:1003B000257500313A2064656C6179282A31306DE9
:1003C00073293A20000A092D2056616C7565732047
:1003D0002D0A004D3E004D25643E20003F00736510
:1003E000742064656661756C740A00433E20000ADF
:1003F000002530325820006B6579626F6172643A73
:100400002000291E1F20212223242526272D2E747B
:100410002A2B141A0815171C180C12132F30280435
:100420001607090A0B0D0E0F3334311D1B06190573
:100430001110363738752C764E4B494C52504F516F
:100440004A4D56545F6061555C5D5E57595A5B6713
:1004500062666377444568696A80707172738080F0
:10046000038048463A3B3C3D3E3F4041424380800A
:1004700080807939007A7880807B7F658080807D7C
:100480008080290A002575002F002575005D280051
:10049000256400200025640020002564002000253C
:1004A00064007C0025303258006D6F7573656B6594
:1004B00079205B62746E7C782079207620685D28D4
:1004C0007265702F61636C293A205B000A092D2048
:1004D0004D61676963202D0A643A09646562756736
:1004E0000A783A096465627567206D61747269788B
:1004F0000A6B3A096465627567206B6579626F61A2
:1005000072640A6D3A096465627567206D6F757370
:10051000650A763A0976657273696F6E0A733A09ED
:100520007374617475730A633A09636F6E736F6CE9
:1005300065206D6F64650A302D343A096C61796508
:1005400072302D34284631302D4634290A506175D9
:10055000733A09626F6F746C6F616465720A000AA6
:10056000092D20436F6E736F6C65202D0A45534330
:100570002F713A09717569740A6D3A096D6F757357
:10058000656B65790A003F0074696D65725F72651D
:100590006164333228293A202530346C580A006BC4
:1005A0006579626F6172645F69646C653A20255891
:1005B0000A006B6579626F6172645F70726F746F4D
:1005C000636F6C3A2025580A00686F73745F6B651F
:1005D00079626F6172645F6C65647328293A2025C3
:1005E000580A000A092D20537461747573202D0A6E
:1005F000004743433A20372E332E30204156522DA8
:100600004C4942433A20322E302E30204156525F20
:10061000415243483A2061767233350A004F5054B4
:10062000494F4E533A204C554641204D4F55534566
:100630004B45592045585452414B455920434F4E44
:10064000534F4C4520434F4D4D414E44204B45594F
:100650004D41505F53454354494F4E203430393655
:100660000A004255494C443A2063313638653220FD
:100670002831353A34323A3532204A756E203138D5
:100680002032303233290A005649443A2030784625
:1006900045454428742E6D2E6B2E29205049443A2E
:1006A000203078393830312850433938206B65791B
:1006B000626F61726420636F6E7665727465722911
:1006C000205645523A203078303130310A004445C6
:1006D00053433A20636F6E766572747320504339CA
:1006E00038206B6579626F6172642070726F746F0D
:1006F000636F6C20696E746F205553420A000A09BB
:100700002D2056657273696F6E202D0A000A6D6F79
:100710007573653A206F66660A000A6D6F757365BA
:100720003A206F6E0A000A6B6579626F6172643AF3
:10073000206F66660A000A6B6579626F6172643ABF
:10074000206F6E0A000A6D61747269783A206F66D4
:10075000660A000A6D61747269783A206F6E0A0049
:100760000A64656275673A206F6E0A000A64656202
:1007700075673A206F66660A000A0A626F6F746CCA
:100780006F616465722E2E2E2000433E20006D6B3B
:100790005F776865656C5F74696D655F746F5F6DC9
:1007A0006178203D2025640A006D6B5F7768656580
:1007B0006C5F6D61785F7370656564203D202564B2
:1007C0000A006D6B5F74696D655F746F5F6D617852
:1007D000203D2025640A006D6B5F6D61785F73704A
:1007E000656564203D2025640A006D6B5F696E7449
:1007F000657276616C203D2025640A006D6B5F6434
:10080000656C6179203D2025640A006D6B5F776817
:1008100065656C5F74696D655F746F5F6D6178208D
:100820003D2025640A006D6B5F776865656C5F6DC0
:1008300061785F7370656564203D2025640A006DF2
:100840006B5F74696D655F746F5F6D6178203D20CB
:1008500025640A006D6B5F6D61785F737065656418
:10086000203D2025640A006D6B5F696E74657276A9
:10087000616C203D2025640A006D6B5F64656C61CE
:1008800079203D2025640A007768657265206465DB
:100890006C74613A20637572736F723D25642C200D
:1008A000776865656C3D25640A53656520687474D6
:1008B000703A2F2F656E2E77696B69706564696178
:1008C0002E6F72672F77696B692F4D6F7573655F38
:1008D0006B6579730A000A092D204D6F7573656B7E
:1008E0006579202D0A4553432F713A097175697452
:1008F0000A313A0964656C6179282A31306D7329AF
:100900000A323A09696E74657276616C286D7329D2
:100910000A333A096D61785F73706565640A343A29
:100920000974696D655F746F5F6D61780A353A09A6
:10093000776865656C5F6D61785F73706565640A83
:10094000363A09776865656C5F74696D655F746FC9
:100950005F6D61780A0A703A097072696E74207668
:10096000616C7565730A643A097365742064656621
:1009700061756C74730A75703A092B310A646F776C
:100980006E3A092D310A706775703A092B31300AB9
:100990007067646F776E3A092D31300A0A7370659B
:1009A0006564203D2064656C7461202A206D617847
:1009B0005F7370656564202A2028726570656174B4
:1009C000202F2074696D655F746F5F6D6178290AEF
:1009D000004C25640A0011241FBECFEFD4E0DEBF17
:1009E000CDBF04B603FE28C08091550490915604F3
:1009F000A0915704B09158048730904BA740B04B5A
:100A0000D9F4109255041092560410925704109283
:100A1000580414BE0FB6F894A895809160008861C0
:100A200080936000109260000FBE10920108109237
:100A30000008E0E0F8E3099511E0A0E0B1E0EEE69F
:100A4000F4E402C005900D92A233B107D9F724E077
:100A5000A2E3B1E001C01D92A535B207E1F70E9403
:100A6000011D0C9435220C940000FF93EF93E0914C
:100A70003201F0913301309709F00995EF91FF9120
:100A80000895FC018591803011F0EFDFFBCF0895D0
:100A9000FF27E0E230E247FF0CC0419597FF09C015
:100AA000EDE26095709580959095611D711D811D99
:100AB000911D27FF02C0219530E350E2AA27660F5F
:100AC000771F881F991FAA1FA41710F0A41B6395F6
:100AD0005A95A9F7AA3008F0A95FA05DAF93F395E6
:100AE000611571058105910541F7ED3211F4EF9320
:100AF000F395F21718F43F93F395FBCF8F91B5DF81
:100B0000FA95E1F70895E991F9918591803021F006
:100B1000853219F0AADFF9CF089520E0E8945591C5
:100B20005532C1F3503311F4689455915A3348F457
:100B3000505390F3220F022E220F220F200D250F6B
:100B4000F4CF0EF4219589919991533619F35337C7
:100B500029F1533559F1BC0188279927E8945C366F
:100B600021F48991999168945591543639F446EF5E
:100B70007EF077FF0DC08FEF9FEF0AC055374AE038
:100B800039F0583540E121F0523642E009F008953D
:100B9000FF93EF937DDFEF91FF91B7CFFF93EF933B
:100BA000FC0181918030B9F360DFFBCFFF93EF93BD
:100BB00068DFF1CFDF93CF93CDB7DEB72596A3DF04
:100BC000CF91DF91089580913F0480FF0CC0609128
:100BD000130170E0759567957595679561157105B9
:100BE00059F1862F089581FF06C06091130170E0CE
:100BF00075956795F3CF6091130170E082FD0CC08D
:100C0000609140046623A9F02091120180911301A4
:100C100090E0621730F0BC0160387105F8F28FE7A0
:100C2000089570E00E94F621622F70E00E94072272
:100C3000F3CF61E070E0D5CF81E0089580913F046B
:100C400080FF11C08091150190E065E070E00E9486
:100C5000F621959587959595879580389105B0F5FE
:100C60000097B1F1089581FF0AC08091150190E0CD
:100C700065E070E00E94F62195958795EECF82FFA2
:100C800008C08091150190E065E070E00E94F621B7
:100C9000E4CF309140043323B1F0209114018091CE
:100CA000150190E065E070E00E94F621BC0132176A
:100CB000A0F6832F90E00E94F621622F70E00E9440
:100CC0000722CB01CACF85E090E008958FE7089511
:100CD00081E00895E72FF0E093E0EE0FFF1F9A9573
:100CE000E1F7E60FF11DEE5FFB4F6491E62FE29511
:100CF000E77090E023E0880F991F2A95E1F78E0FA7
:100D0000911D34E0880F991F3A95E1F7E62FEF70B7
:100D1000E80FF92FF11DEE0FFF1FE050F849859104
:100D2000949108952FB7F89480914A0490914B04C0
:100D3000A0914C04B0914D042FBF0895E4E3F2E07C
:100D40009281891301C01282319692E0EA33F90749
:100D5000B9F70895A6E3B2E0EFEF90E02D91821786
:100D600051F0EF3F19F4211101C0E92F9F5F963038
:100D7000A9F7EF3F09F408950E2E000CFF0BEC5C71
:100D8000FD4F828308954F925F926F927F929F9260
:100D9000AF92BF92CF92DF92EF92FF920F931F9389
:100DA000CF93DF9300D000D01F92CDB7DEB76B8317
:100DB0007C838D837A018C819D81892B49F08FEF13
:100DC000F81204C081E09FEF491719F080E001C0DC
:100DD00081E080FD6AC00F2D10E0CE2CD12C8B81DC
:100DE000882309F456C04090B7035090B803609030
:100DF000B9037090BA038091510490915204A0916C
:100E00005304B0915404482A592A6A2A7B2A2FE1B4
:100E1000A22EB12C9A2CD301C2010A2C04C0B69583
:100E2000A795979587950A94D2F780FD2BC081E00E
:100E3000A81AB10878F7912CF80193E0EE0FFF1F84
:100E40009A95E1F7E554FC4FEC0DFD1D9082E98287
:100E5000FA8269817A81892D0F900F900F900F90FF
:100E60000F90DF91CF911F910F91FF90EF90DF9046
:100E7000CF90BF90AF909F907F906F905F904F907A
:100E80000C946A06B7018A2D0E946A06019779F2CE
:100E9000D3CFF80183E0EE0FFF1F8A95E1F7E55409
:100EA000FC4FEC0DFD1D9080D2CF90E080E00F90C4
:100EB0000F900F900F900F90DF91CF911F910F9196
:100EC000FF90EF90DF90CF90BF90AF909F907F907A
:100ED0006F905F904F90089541E050E060E070E0C7
:100EE00004C0440F551F661F771F8A95D2F740959F
:100EF0005095609570958091B7039091B803A0913B
:100F0000B903B091BA0384239523A623B723809312
:100F1000B7039093B803A093B903B093BA030895AD
:100F200041E050E060E070E004C0440F551F661FD0
:100F3000771F8A95D2F78091B7039091B803A0915B
:100F4000B903B091BA03842B952BA62BB72B8093B2
:100F5000B7039093B803A093B903B093BA0308956D
:100F60008091B60390918503981301C008958F5F17
:100F70008770FACF1F93CF93DF9300D000D01F92DA
:100F8000CDB7DEB7942F4983252F5A836B837C839B
:100F90008D834C815D8181E0452B31F02F3F19F429
:100FA00081E09F3F09F080E0182F117080FD2CC078
:100FB00049815A816B817C818D810E94C306292FD2
:100FC00022952F702C3078F42A30A8F42250223049
:100FD000C8F0812F0F900F900F900F900F90DF911E
:100FE000CF911F9108952C3011F02F3091F793FB82
:100FF000112710F9EECF803C28F0803E50F3815F3E
:10100000833038F311E0E5CF10E0E3CFE091410405
:10101000F0914204309721F00190F081E02D099485
:1010200080E008951092E2001092E100E0EEF0E01E
:10103000808181608083E8EDF0E080818F7780831C
:1010400019BCE3E6F0E08081816080831092530355
:1010500008950E941208F89487E797E79093010893
:101060008093000887E090EBDC0180935504909317
:101070005604A0935704B093580488E19CE00FB63F
:10108000F894A895809360000FBE90936000FFCF06
:10109000FC01809167039091680386179707A0F081
:1010A0006115710529F49091E8009E779093E8000E
:1010B00090E06115710551F4911108C08091E8002C
:1010C00082FF32C080E00895BC01F2CF80916903B5
:1010D0008823B1F18530B1F18091E80083FD2EC005
:1010E0008091E80082FDEACF8091E80080FFE1CFA7
:1010F0002091F20030E06115710519F028303105BA
:1011000058F091E02830310509F090E02091E80096
:101110002E772093E800CDCF81918093F10061502C
:1011200071092F5F3F4FE7CF80916903882341F01A
:10113000853041F08091E80083FFC0CF81E00895C1
:1011400082E0089583E008952091E4003091E50065
:1011500085E69091EC0090FF06C09091E80090FF2A
:1011600006C080E008959091E80092FDFACF90913A
:101170006903992391F0953091F09091EB0095FDE2
:1011800010C04091E4005091E5002417350709F3A1
:1011900081509A01F1F684E0089582E0089583E099
:1011A000089581E008958091610387FF13C08091C5
:1011B000E80082FF06C08091E8008B778093E8000A
:1011C00004C0809169038111F2CF08958091690371
:1011D0008823D9F38091E80080FFF8CF8091E80060
:1011E0008E77ECCF982F9093E900242F762F50E044
:1011F000891731F07091EC002091ED005091F000D2
:1012000021FD07C09F5F953071F78093E90081E071
:1012100008953091EB003E7F3093EB003091ED006C
:101220003D7F3093ED003091EB0031603093EB0067
:101230007093EC002093ED005093F0002091EE00AD
:1012400027FDE0CF80E008950F931F93CF93DF93A6
:10125000CDB7DEB7AA970FB6F894DEBF0FBECDBFED
:1012600080916903882309F44EC11091E9001F7031
:101270008091EC0080FF39C080E8182B1092E900C3
:101280008091E80083FF3CC1E1E6F3E089E693E06A
:101290002091F10021938E179F07D1F7809162036F
:1012A000833009F470C018F5813009F447C08230EA
:1012B00009F4DAC08091E80083FF14C180916103D2
:1012C000909162039A3008F00DC1E92FF0E0E559E2
:1012D000F64F0C941B22450A6B0A720A6B0A720ABB
:1012E000CD0AEF0A720AEA0BF70B80E0C6CF8A300C
:1012F00009F4A9C08B3009F47DC08930D9F68091FA
:1013000061038132B9F68091650390916603892B60
:1013100089F68091E800877F8093E8008091E8005B
:1013200082FF2CC08091F100809355038091E800EA
:101330008B778093E8000E94D308BCCF8091610333
:10134000813A09F0B7CF8091E800877F8093E80069
:101350008091650390916603892B61F060E090E0D5
:1013600080E070E00E9448088091E8008B778093CD
:10137000E800A0CF68E086E593E0F3CF80916903B1
:101380008111CCCF97CF80916103813A09F092CF40
:101390008091650390916603892BA1F48091E80008
:1013A000877F8093E8008091E80080FFFCCF8091E8
:1013B00011018093F1008091E8008E778093E8001E
:1013C0000E94D3088091650390916603019709F00C
:1013D00071CF8091E800877F8093E8008091E800DA
:1013E00080FFFCCF809110018093F1008091E80094
:1013F0008E779FCF80916103813209F05BCF80911E
:10140000650390916603892B59F48091E800877FEA
:101410008093E8000E94D3088091630380931101B8
:101420008091650390916603019709F043CF809105
:10143000E800877F8093E8000E94D30880916303CF
:101440008093100137CF80916103813209F032CF50
:101450008091E800877F8093E8000E94D308809104
:10146000640380934E0426CF80916103813A09F092
:1014700021CF8091E800877F8093E8008091E80089
:1014800080FFFCCF80914E04AFCF803889F0823846
:1014900049F5809165038F70853020F58093E900D0
:1014A0008091EB0085FB882780F91092E90006C047
:1014B00080915E0390915F03911182609091E800AA
:1014C000977F9093E8008093F1001092F100809153
:1014D000E8008E7731C0282F2D7F21F48823F1F08A
:1014E000823079F18091E80083FF0AC08091E800A2
:1014F000877F8093E8008091EB0080628093EB000F
:101500001F701093E900AA960FB6F894DEBF0FBEC5
:10151000CDBFDF91CF911F910F910895809163030B
:10152000813001F7933009F080E080935F031092DF
:10153000E9008091E800877F8093E8000E94D3084B
:10154000D1CF809163038111F2CF809165038F70B9
:101550002FEF280F243030F68093E9002091EB0024
:1015600020FFE5CF933031F48091EB0080628093CF
:10157000EB00DDCF9091EB0090619093EB0021E0C8
:1015800030E001C0220F8A95EAF72093EA0010921A
:10159000EA008091EB008860EACF8111A3CF00912F
:1015A00063030F778091E3008078802B8093E300C2
:1015B0008091E800877F8093E8000E94D3088091A3
:1015C000E80080FFFCCF8091E30080688093E30017
:1015D00083E0011101C082E08093690383CF8058CA
:1015E000823008F07FCF20916303309164032C3D5B
:1015F00083E03807A1F583E08A838AE289834FB7C5
:10160000F894DE01139620E03EE051E2E32FF0E093
:1016100050935700E49120FF03C0E295EF703F5FC5
:10162000EF708E2F90E0EA30C0F0C7968D939D93B7
:101630002F5F243159F74FBF8091E800877F809357
:10164000E8006AE270E0CE0101960E9448088091AD
:10165000E8008B778093E80045CFC096E7CF809174
:10166000650390916603432F55274330510509F4D4
:101670004FC078F54130510509F445C084E590E04C
:10168000E3E6F2E04230510509F02CCF2091E8006A
:10169000277F2093E8002091670330916803821729
:1016A000930708F49C0140E02115310509F063C05F
:1016B000411161C08091E80082FDC9CF809169032A
:1016C000882329F2853019F28091E80083FFF2CF58
:1016D000BECF4132510509F43FC04232510509F0F5
:1016E00001CF8330910508F0FDCEFC01EE0FFF1F06
:1016F000E45EFE4F0190F081E02D875E9E4FDC019D
:101700008C9190E01DC082E190E0E7EBF2E0BECF6B
:10171000332721303105C1F060F02230310509F066
:10172000E1CEE9ECF2E0E4918E2F90E0E9ECF2E01A
:1017300007C0EBE0F3E0E4918E2F90E0EBE0F3E004
:10174000009709F4CFCEA2CFEBEFF2E0E4918E2F19
:1017500090E0EBEFF2E0F4CF8330910508F0C2CED9
:10176000880F991FFC01EE5DFE4F0190F081E02D86
:1017700089E090E08BCF80916903882309F467CFDB
:10178000853009F464CF8091E80083FD60CF8091BB
:10179000E80082FD8FCF8091E80080FF85CF8091A7
:1017A000F20090E02115310519F08830910550F0D4
:1017B00041E0089709F040E08091E8008E7780933F
:1017C000E80072CF44914093F100319621503109E5
:1017D0000196E8CF803809F085CE8091E800877FB8
:1017E0008093E800809160038093F10070CE8111B6
:1017F00079CE00916303023008F074CE8091E80046
:10180000877F8093E800009360030E94D308002341
:1018100099F084E08093690342E061EC81E00E94EA
:10182000F20842E061EC82E00E94F20846E261ECDC
:1018300083E00E94F20856CE8091E30087FDE9CF55
:1018400081E0E8CFEF92FF920F931F93CF937C013B
:101850008B010E94A408C82F811119C08091E80053
:1018600085FD0DC08091E8008E778093E8000E948E
:1018700024090E94A408882389F3C82F08C0F7010F
:1018800081917F018093F1000150110939F78C2F6C
:10189000CF911F910F91FF90EF9008958091550384
:1018A000089580913E03811113C09FB7F894409131
:1018B0004A0450914B0460914C0470914D049FBFB9
:1018C000443C59406105710518F081E080933E0366
:1018D0000895EF92FF920F931F93CF93DF93D82F2A
:1018E0000FB607FE46C080916903843079F080917D
:1018F000030190E001962091050130E082239323BB
:10190000209104012817190609F0C9C00E94510C42
:1019100081110FC08091030190E001962091050193
:1019200030E082239323209104012817190609F03F
:10193000B6C00E9492068C01C091E900CF708091E0
:10194000EC0080FD37C080E0C82B83E08093E90085
:1019500085E0E82E8091EB0085FD08C08091EB00CA
:1019600080FF04C08091EE0087FD44C0CF70C0931B
:10197000E900E09103018E2F90E00196209105018E
:1019800030E082239323209104012817190609F4DB
:101990007EC08091010190910201E80FF92FF11DA5
:1019A000D083809103018F5F9091050189238093FB
:1019B00003016DC080E8C8CFE0910101F091020100
:1019C000E80FF11D90818F5F2091050182238093A4
:1019D00004019093F1008091E80085FD0BC0809197
:1019E000E80080FF07C08091E8008E778093E800D0
:1019F000E09200018091040190910301981741F158
:101A00009091E80095FDD8CF80E029C01092F100B8
:101A10002EC08091030190E001962091050130E0F5
:101A200082239323209104012817190609F09ECFE1
:101A3000F0900001FF2009F499CF0E9492068017D0
:101A4000910709F487CFFA94F09200018C0182CFBC
:101A50008091E80085FFD8CFD093F10081E090918C
:101A6000F200992379F09091E80090FF0BC09091DB
:101A7000E80095FDCBCF9091E8009E779093E80029
:101A8000E0920001882329F2CF70C093E90080E042
:101A9000DF91CF911F910F91FF90EF900895E0910A
:101AA000030177CF90913C0380913D03891751F05A
:101AB000E92FF0E0E45CFD4F80819F5F90933C0351
:101AC00090E008958FEF9FEF08958330C9F128F4D7
:101AD000813061F0823019F10895853009F452C0E7
:101AE00008F43FC0863009F45EC008958091170164
:101AF000681790F4861B80931701809117011F923D
:101B00008F9389E798E09F938F930E94DA050F9057
:101B10000F900F900F90089510921701EECF8091C3
:101B20001601681750F4861B8093160180911601E8
:101B30001F928F9387E698E0E6CF10921601F6CFBA
:101B400080911501681750F4861B809315018091D0
:101B500015011F928F9384E598E0D5CF109215015F
:101B6000F6CF80911401681750F4861B80931401FE
:101B7000809114011F928F938FE398E0C4CF10924D
:101B80001401F6CF80911301681750F4861B8093DF
:101B90001301809113011F928F9386E298E0B3CFD7
:101BA00010921301F6CF80911201681750F4861B32
:101BB00080931201809112011F928F938BE098E025
:101BC000A2CF10921201F6CF833009F445C028F459
:101BD000813061F0823049F10895853009F46AC09E
:101BE00008F451C0863009F47CC008958091170133
:101BF000482F460F5527551F4F3F510594F4680F46
:101C000060931701809117011F928F938CEF97E0DB
:101C10009F938F930E94DA050F900F900F900F9073
:101C200008958FEF80931701EDCF80911601482F13
:101C3000460F5527551F4F3F510554F4680F6093C9
:101C40001601809116011F928F938AEE97E0E0CFE4
:101C50008FEF80931601F5CF80911501482F460F25
:101C60005527551F4F3F510554F4680F60931501D8
:101C7000809115011F928F9387ED97E0C9CF8FEF69
:101C800080931501F5CF80911401482F460F5527F9
:101C9000551F4F3F510554F4680F60931401809114
:101CA00014011F928F9382EC97E0B2CF8FEF809355
:101CB0001401F5CF80911301482F460F5527551F6A
:101CC0004F3F510554F4680F609313018091130145
:101CD0001F928F9389EA97E09BCF8FEF8093130138
:101CE000F5CF80911201482F460F5527551F4F3FC2
:101CF000510554F4680F60931201809112011F92F4
:101D00008F938EE897E084CF8FEF80931201F5CF09
:101D1000CF93DF9320916C0330916D03281739071F
:101D200001F190936D0380936C03E0914104F09175
:101D300042043097B1F0EC010084F185E02D099563
:101D4000809150048570853061F4DF93CF938DE1ED
:101D500093E09F938F930E94DA050F900F900F905E
:101D60000F90DF91CF910895CF93DF9320916A0375
:101D700030916B032817390701F190936B0380931F
:101D80006A03E0914104F09142043097B1F0EC0114
:101D90000680F781E02D099580915004857085308B
:101DA00061F4DF93CF938FE093E09F938F930E9432
:101DB000DA050F900F900F900F90DF91CF9108955B
:101DC00086ED98E00E9441051F9281E08F931F925B
:101DD00085E08F9388E898E09F938F930E94DA05BF
:101DE0000F900F900F900F900F900F900895CF933A
:101DF0008091500483FF7EC089EA94E00E944105EF
:101E0000809145041F928F9384EA94E09F938F936F
:101E10000E94DA0582EA94E00E944105809146041E
:101E2000282F082E000C330B3F938F938FE994E0FB
:101E30009F938F930E94DA058DE994E00E944105FB
:101E400080914704282F082E000C330B3F938F936B
:101E50008AE994E09F938F930E94DA0588E994E0E1
:101E60000E94410580914804282F082E000C330B56
:101E70003F938F9385E994E09F938F930E94DA05B7
:101E800083E994E00E94410580914904282F082E9F
:101E9000000C330B3F938F9380E994E09F938F93D3
:101EA0000E94DA058DE894E00E944105809140048B
:101EB0001F928F938AE894E09F938F930E94DA0594
:101EC00088E894E00E94410580913F041F928F931F
:101ED00085E894E09F938F930E94DA0582E894E06E
:101EE0000E9441058DB79EB74C960FB6F8949EBFE1
:101EF0000FBE8DBFE0914104F0914204309751F044
:101F0000C09145040480F581E02D85E494E00995B5
:101F1000C09345040E949206909344048093430426
:101F2000CF9108950F931F93CF93DF9380913D043A
:101F300090913C04892B8093340290913B04992327
:101F400089F0892B80933402E5E3F2E02CE332E060
:101F500080E0919191118F5F2E173F07D1F781118A
:101F600010923B04E0914104F09142043097B1F1AA
:101F70000280F381E02D84E392E009958091500482
:101F800082FF2CC080FF04C087EF93E00E944105D0
:101F9000D0E0C0E001EF13E08091500480FF0EC05C
:101FA000FE01EC5CFD4F80811F928F931F930F9376
:101FB0000E94DA050F900F900F900F902196C83075
:101FC000D10551F78091500480FF08C08FEE93E057
:101FD000DF91CF911F910F910C944105DF91CF912B
:101FE0001F910F91089510923D0410923C04E4E378
:101FF000F2E01182128213821482158216821782F5
:102000000E94920F85E0E5E4F4E0DF011D928A95DD
:10201000E9F71092400410923F040E94F70E90E0FE
:1020200080E00E94B40E90E080E00C94880ECF9384
:10203000C82F1F928F9381ED99E09F938F930E94F9
:10204000DA0581E090E0A0E0B0E004C0880F991FBD
:10205000AA1FBB1FCA95D2F78093510490935204D4
:10206000A0935304B09354040F900F900F900F90CF
:10207000CF910C94F30F882341F0809590913D040B
:10208000892380933D040C94920F0895882339F09E
:1020900090913D04892B80933D040C94920F0895F8
:1020A0008732D8F58E3108F0FCC08E3009F48FC02D
:1020B00078F4873009F470C08B3009F456C086304C
:1020C00009F458C086E895E00E94410580E0089533
:1020D000863109F4A6C078F48031A1F790915004BC
:1020E000892F877F93FF88608093500483FF7FC090
:1020F0008AE197E063C0893109F47CC08B3111F724
:1021000090915004892F8D7F91FF826080935004BD
:1021100081FF5AC083E597E051C0883331F150F414
:10212000893221F0853311F0873261F680E00E9418
:10213000171040C08334D1F320F48A3318F2895346
:10214000F6CF883409F0BECF0E94F30F89E797E0FD
:102150000E9441052FEF83ED90E321508040904095
:10216000E1F700C000000E9429088CEC94E00E9476
:10217000410520C080915004817F8E7F8093500460
:102180008FE595E00E9441058AE897E00E944105AD
:1021900081E080934F0408958091500480FF0CC02B
:1021A0008CE697E00E94410580915004817F8E7FEC
:1021B0008093500481E0089580E697E00E944105F5
:1021C000809150048160F4CF85E497E0D0CF909166
:1021D0005004892F8B7F92FF84608093500482FF8C
:1021E00003C086E397E0EACF86E297E0C0CF8DE0B8
:1021F00097E0BDCF8EEF96E00E9441058EEC96E011
:102200000E94410588E896E00E94410582E696E03A
:102210000E9441058DE196E00E94410581EF95E025
:10222000A6CF83EE95E00E9441050E9406081F920A
:102230008F9389EC95E09F938F930E94DA058091AC
:1022400011011F928F9382EB95E09F938F930E94D1
:10225000DA0580914E041F928F938FE995E09F934A
:102260008F930E94DA052FB7F89480914A049091D9
:102270004B04A0914C04B0914D042FBFBF93AF937A
:102280009F938F9388E895E09F938F930E94DA0540
:102290008DB79EB742960FB6F8949EBF0FBE8DBF06
:1022A00089CF8D5144CFCF93DF93882309F454C055
:1022B0009EE7980F933020F5C2E0D9E3823831F0E1
:1022C000C4E0D7E4833811F4C1E0D3E50E940608E6
:1022D0008C2309F441C08D2F0E94AA060E94920F00
:1022E0002FEF41EE54E0215040405040E1F700C054
:1022F00000008D2F0E949E06DF91CF910C94920FCB
:102300009CEF980F913AB0F390E2980F983088F4D0
:10231000877021E030E0A90102C0440F551F8A9563
:10232000E2F7CA01809590913D04892380933D0492
:10233000E3CF9BE5980F933030F490E080E0DF919D
:10234000CF910C94B40E885A873130F490E080E03D
:10235000DF91CF910C94880EDF91CF910895CF93A8
:10236000DF93882309F4C6C0C82F8EE78C0F833013
:1023700030F5C238F1F0C338F9F0C4E0D7E40E9478
:1023800006088C2309F0B6C08D2F0E94AA060E9471
:10239000920F2FEF81EE94E0215080409040E1F7C2
:1023A00000C000008D2F0E949E06DF91CF910C94FB
:1023B000920FC2E0D9E3E3CFC1E0D3E5E0CF8CEFE9
:1023C0008C0F813A08F043C180914F048130C1F0F5
:1023D00048F0823009F445C010924F048C2F0E94BF
:1023E000AA06E3CF80917A0380FD04C08091340275
:1023F0008434A1F78C2F0E94501081117BC0EECF46
:1024000080917A0380FDF6CF80913402843491F379
:10241000C431C9F048F4CB3059F0C031C1F08DE27D
:1024200093E00E94410511C0C93269F0C833B9F781
:102430008FE595E00E94410583E393E00E9441050A
:1024400081E08170DACF10924F0480E0FACF0E94D1
:10245000E00E8FE293E00E94410582E080934F04FA
:10246000EFCFC432D0F4CE3108F0C0C0CB30E9F0A9
:1024700048F4C73009F4D1C08CED93E0DF91CF91DF
:102480000C944105C331C9F1C431B1F780917E0389
:10249000882349F110927E030AC0CB3409F4BBC0F3
:1024A000C0F4C93299F3C83339F70E94E00E809125
:1024B0007E03882309F4C8C01F928F9386ED93E0B2
:1024C0009F938F930E94DA050F900F900F900F90BB
:1024D00011C0C13509F499C0C23509F490C0CE3499
:1024E00059F66AE093C08BEE93E00E94410581E0CB
:1024F00080934F04DF91CF91089585EC93E00E9483
:10250000410583EB93E00E944105809117011F92E2
:102510008F9380EB93E09F938F930E94DA058EEA6E
:1025200093E00E9441058CE993E00E94410580916F
:1025300016011F928F9389E993E09F938F930E94D6
:10254000DA0587E993E00E94410588E893E00E945C
:102550004105809115011F928F9385E893E09F9329
:102560008F930E94DA0583E893E00E94410582E799
:1025700093E00E944105809114011F928F938FE692
:1025800093E09F938F930E94DA058DE693E00E947B
:10259000410588E593E00E944105809113011F9257
:1025A0008F9385E593E09F938F930E94DA0583E5EF
:1025B00093E00E9441058CE393E00E9441058091E5
:1025C00012011F928F9389E393E09F938F930E9450
:1025D000DA0587E393E00E9441058DB79EB74896E0
:1025E0000FB6F8949EBF0FBE8DBF61CFCE51EC2FBA
:1025F000F0E0E85DFE4F808180937E0358CF61E07C
:1026000080917E030E94E40D52CF61E080917E03B1
:102610000E94650D4CCF6AE0F3CF8EE180931701E5
:1026200082E3809316018AE08093150184E1809310
:10263000140188E08093130188E2809312018EEDEB
:1026400093E00E94410533CF83ED93E017CF80E202
:102650008C0F883068F4C77021E030E001C0220F91
:10266000CA95EAF780913D04822B80933D049DCE6C
:102670008BE58C0F833070F481E890E0C53A31F03F
:1026800083E890E0C63A11F482E890E0DF91CF91C0
:102690000C94B40E88E58C0F873108F069C082EE87
:1026A00090E0C83A09F460C089EE90E0C93A09F4B4
:1026B0005BC08AEE90E0CA3A09F456C085EB90E020
:1026C000CB3A09F451C086EB90E0CC3A09F44CC007
:1026D00083EB90E0CD3A09F447C084EB90E0CE3A2A
:1026E00009F442C087EB90E0CF3AF1F18CEC90E036
:1026F000C13BD1F18DEC90E0C03BB1F183E891E0BA
:10270000C23B91F18AE891E0C33B71F182E991E02B
:10271000C43B51F184E991E0C53B31F181E292E0A3
:10272000C63B11F183E292E0C73BF1F084E292E014
:10273000C83BD1F085E292E0C93BB1F086E292E07D
:10274000CA3B91F087E292E0CB3B71F08AE292E0E3
:10275000CC3B51F08FE690E0CD3B31F090E080E053
:10276000CE3B11F480E790E0DF91CF910C94880E7E
:10277000CF3B09F0BFCE0E94F30F9FEF20E782E02E
:10278000915020408040E1F700C000000E942908DD
:10279000CF92DF92EF92FF920F931F93CF93DF932D
:1027A00000D000D01F92CDB7DEB76C0185E0F601F6
:1027B000DE01119601900D928A95E1F7F6014081B4
:1027C00051812381348191E02115310531F05F3F42
:1027D00019F491E04F3F09F090E090FD99C0F601A7
:1027E0000281F580F2949FE0F92249835A830B839A
:1027F000722F3D832C83602F8D810E94C306182F7A
:10280000E92FE295EF70EF3008F082C0F0E0E55F6D
:10281000FB4E0C941B221A141A1458145814CE147C
:10282000001588148814F2158814C816C816881460
:1028300088148417F92FFF70FF2E907F19F0F294FF
:1028400080EFF8220023C9F0FF2039F080913C048A
:10285000F82AF0923C040E94920F812F0F900F9063
:102860000F900F900F90DF91CF911F910F91FF90DC
:10287000EF90DF90CF900C94AF11812F0E945311F5
:10288000FF2009F445C0F09480913C04F822F092B6
:102890003C040F900F900F900F900F90DF91CF910D
:1028A0001F910F91FF90EF90DF90CF900C94920FBB
:1028B000892F8F70907F903211F08295807F112345
:1028C00079F0113009F449C0002309F455C0FF2004
:1028D00059F0F601958190FF69C29F70958304C0FD
:1028E000002321F1F1100FC00F900F900F900F9067
:1028F0000F90DF91CF911F910F91FF90EF90DF909C
:10290000CF900C94461021E0F212EECF80933B045E
:102910000F900F900F900F900F90DF91CF911F911C
:102920000F91FF90EF90DF90CF900895F11011C0BC
:1029300010923B040F900F900F900F900F90DF912B
:10294000CF911F910F91FF90EF90DF90CF900C945B
:102950003B1091E0F912ECCFDBCF002349F0E5E02A
:10296000EF15B0F290913D04982309F4BDCFE2CF6A
:10297000F4E0FF1568F2DECFFF20E1F2812F0F9027
:102980000F900F900F900F90DF91CF911F910F91AB
:10299000FF90EF90DF90CF900C945311892F869584
:1029A00086958370C1F0813009F0B2CF812F93708A
:1029B000011102C090E080E00F900F900F900F90F7
:1029C0000F90DF91CF911F910F91FF90EF90DF90CB
:1029D000CF900C94880E812F9370011102C090E06B
:1029E00080E00F900F900F900F900F90DF91CF919C
:1029F0001F910F91FF90EF90DF90CF900C94B40E49
:102A0000002309F471C0803FA1F40E941E06819545
:102A1000809347040F900F900F900F900F90DF91CD
:102A2000CF911F910F91FF90EF90DF90CF900C947A
:102A3000F70E813F19F40E941E06EACF823F31F45F
:102A40000E941E06819580934604E4CF833F19F4CB
:102A50000E941E06F8CF893F29F40E94E305809367
:102A60004804D8CF8A3F21F40E94E3058195F7CF2F
:102A70008B3F31F40E94E305819580934904CACFCE
:102A80008C3F19F40E94E305F8CF809145048160E2
:102A9000143FA1F0809145048260153F79F0809148
:102AA00045048460163F51F0809145048860173FCB
:102AB00029F0183F31F480914504806180934504EA
:102AC000A9CF80913F0481601D3F59F080913F0460
:102AD00082601E3F31F01F3F09F09CCF80913F0480
:102AE000846080933F0496CF803FC1F48091470477
:102AF00087FD109247048091460481118BCF80910D
:102B00004704811187CF80914804811183CF809140
:102B1000490481117FCF109240047CCF813F29F47A
:102B20008091470418162CF3E6CF80914604123F9B
:102B300029F487FFE0CF10924604DDCF133F19F44C
:102B40001816CCF3D8CF193F39F4809148041816E1
:102B500094F610924804CFCF1A3F29F4809148048C
:102B600087FFC9CFF6CF1B3F39F48091490487FF17
:102B7000C2CF10924904BFCF1C3F29F48091490471
:102B80001816BCF3B8CF809145048E7F143FA1F096
:102B9000809145048D7F153F79F0809145048B7FAE
:102BA000163F51F080914504877F173F29F0183F69
:102BB00031F4809145048F7E809345049CCF8091B1
:102BC0003F048E7F1D3F59F080913F048D7F1E3F53
:102BD00031F01F3F09F08FCF80913F048B7F8093AE
:102BE0003F0489CF892F837009F064C0011190CE12
:102BF000812F829586958770880F880F412F4F709F
:102C0000C42ED12CF12CE12C082E04C0CC0CDD1CE0
:102C1000EE1CFF1C0A94D2F740E050E0BA0114FF0A
:102C200011C00FE010E020E030E004C0000F111FE1
:102C3000221F331F8A95D2F7B901A80140955095FC
:102C400060957095009151041091520420915304A5
:102C5000309154049695969593709230E9F028F54A
:102C6000913089F04C295D296E297F294023512319
:102C7000622373234093510450935204609353048E
:102C80007093540445CEC02AD12AE22AF32A4C2953
:102C90005D296E297F29EECF4C295D296E297F2978
:102CA0004027512762277327E5CF40235123622312
:102CB0007323EDCF8695002311F0892F817088232F
:102CC00009F426CE812F829586958770880F880F0C
:102CD000412F4F70C42ED12CF12CE12C082E04C0B2
:102CE000CC0CDD1CEE1CFF1C0A94D2F740E050E037
:102CF000BA0114FF11C00FE010E020E030E004C082
:102D0000000F111F221F331F8A95D2F7B901A801A6
:102D100040955095609570950091B7031091B80358
:102D20002091B9033091BA0396959695937092309D
:102D3000E9F028F5913089F04C295D296E297F2929
:102D400040235123622373234093B7035093B80366
:102D50006093B9037093BA03DBCD0C291D292E298A
:102D60003F29402B512B622B732BEECF4C295D2931
:102D70006E297F294027512762277327E5CF4023FB
:102D80005123622373234C295D296E297F29DCCFCF
:102D9000803F09F44EC0D0F480E4810F803270F19E
:102DA000002309F4ACC0FF2009F4A6C0812F0E94C3
:102DB000AF11193309F099C0FFEF21EE84E0F15013
:102DC00020408040E1F700C00000A2CD823F09F41E
:102DD00070C008F45BC0833F19F7002309F47CC07E
:102DE000292F2F7181E090E0A0E0B0E004C0880FAF
:102DF000991FAA1FBB1F2A95D2F73AC0E12FE07195
:102E0000FE2E892F8F71002351F00E949007812F91
:102E10008295807FF11068CD812F8F7065CD0E94E3
:102E20006C07812F8295807FF11084CD812F8F7068
:102E300081CD002331F1F4E0FF1508F469CD292F8D
:102E40002F7181E090E0A0E0B0E004C0880F991FEE
:102E5000AA1FBB1F2A95D2F74091B7035091B80320
:102E60006091B9037091BA0384279527A627B727E5
:102E70008093B7039093B803A093B903B093BA03B8
:102E800047CD25E02F1508F443CDD9CF892F8F7179
:102E9000002399F00F900F900F900F900F90DF91FB
:102EA000CF911F910F91FF90EF90DF90CF900C94F6
:102EB0009007892F8F71002369F30F900F900F9067
:102EC0000F900F90DF91CF911F910F91FF90EF9096
:102ED000DF90CF900C946C071092B7031092B80358
:102EE0001092B9031092BA0313CD133509F464CFCD
:102EF000173409F00DCD60CF892F8F71CBCFF11032
:102F00003DCD892F8F71D9CF811102CD002309F4D6
:102F1000FFCC0E94F30F8FEF90E7E2E081509040EA
:102F2000E040E1F700C000000E9429081F93CF9302
:102F3000DF9380918403807FB1F4809181038823A3
:102F400091F02091B60310918503C0917F03D09139
:102F50008003A0918203B091830341E0CF3F09F049
:102F600040E0121304C0DF91CF911F91089581E0DA
:102F7000109721F0842FDF3F09F080E030E080FDE2
:102F800033C0C90166E070E00E94F621FC01EA57F7
:102F9000FC4F81818D1328C080818C1325C08281D4
:102FA000811122C0838194818A1B9B0B883C9105EF
:102FB000D8F4809184038F70806180938403C90169
:102FC00066E070E00E94F621FC01E557FC4F90811D
:102FD0009F70906190838FE793E00E94C813DF9108
:102FE000CF911F910C94B0072F5F3F4F2770B9CF3F
:102FF0009F92AF92BF92CF92DF92EF92FF920F9388
:103000001F93CF93DF93CDB7DEB761970FB6F894D8
:10301000DEBF0FBECDBF8C0185E0F801DE011D963D
:1030200001900D928A95E1F7F80140812181F280AB
:10303000C380D48090917F0330918003609182039C
:103040007091830381E06115710531F03F3F19F400
:1030500081E09F3F09F080E0F82FF1709F2E80FD06
:103060004EC18FE7A82E83E0B82EE0908103F601D1
:10307000E61BF70BEE2009F404C180918403582F5E
:10308000507FE83CF10508F0BDC0511183C0EF2C22
:10309000321322C0941320C0F1101EC08F708061C3
:1030A00080938403C5010E94C81380918403F801B2
:1030B00085838E2D61960FB6F894DEBF0FBECDBF0F
:1030C000DF91CF911F910F91FF90EF90DF90CF9004
:1030D000BF90AF909F90089581E0C114D10431F06A
:1030E0002F3F19F481E04F3F09F080E080FD14C0CC
:1030F00081E08F25F82FF170BF2EE091B60330915B
:10310000850380FD22C0FF20A1F2809184038160AD
:1031100080938403E12CCDCF80E0ECCFF0E0CF01B1
:1031200066E070E00E94F621DC01AA57BC4F1196C0
:103130008C911197281307C08C91481304C01296E4
:103140008C918F11E0CF3196E770E313E7CF7C2DA0
:10315000D98AC88A522F6F2D89890E94C306292FC8
:1031600022952F70223050F0243078F49F7051F067
:10317000F8019581907F31F4E92C9BCF9F7011F07D
:103180008823D1F3805E8830B8F3C8010E94C81349
:103190009B2CF2CF321306C0941304C0F801FF2019
:1031A00009F48AC04D872E87FF867C2DD98AC88A6C
:1031B000522F6F2D89890E94BA07882309F4AEC067
:1031C000FF2009F4ABC080918403803270F020911D
:1031D0007F033091800338872F831986DB86CA8668
:1031E0008C87CE0107960E94C81386E0F801AFE7EE
:1031F000B3E001900D928A95E1F70E949617EE24B4
:10320000E39457CF51110AC08FE793E00E94C8138F
:1032100086E0F50111928A95E9F77CCF32130FC051
:1032200094130DC0F1100BC0F8018583C8010E94F2
:10323000C81386E0F50111928A95E9F73ACF4D87D8
:103240002E87FF867C2DD98AC88A522F6F2D8989B7
:103250000E94BA07882309F461C0FF2009F45EC008
:1032600080918403803208F220917F0330918003A3
:103270003A8329831B82DD82CC828E83CE01019624
:10328000B2CFE83CF105A8F6EF2CFF2009F446C0C8
:1032900032131FC094131DC08091840380FD10C0A1
:1032A000982F907F69F0F8018583903F31F0982F37
:1032B000907F905F8F70892B8583C8010E94C8130F
:1032C00086E0F801AFE7B3E001900D928A95E1F74F
:1032D000F0CE4D872E87FF867C2DD98AC88A522F43
:1032E0006F2D89890E94BA0781117FCF8091840355
:1032F000816080938403C8010E94C813DACEFF2046
:1033000069F04D872E87FF867C2DD98AC88A522F77
:103310006F2D89890E94BA07811167CFC8010E9469
:10332000C8136DCFCF93DF93CDB7DEB767970FB6D6
:10333000F894DEBF0FBECDBF4B8B5C8B6D8B7E8B4D
:103340008F8B1A8A198A85E0FE017396DE011D961D
:1033500001900D928A95E1F786E0FE013D96DE012F
:10336000179601900D928A95E1F7CE0107960E947B
:10337000F817811138C086E0FE013796DE011196FC
:1033800001900D928A95E1F79F8188852A853B857A
:10339000232B39F08F3F19F481E09F3F19F080E033
:1033A00001C081E080FD1FC08091850390E09C01F9
:1033B0002F5F3F4F277033274091B6034217130604
:1033C00061F166E070E00E94F621DC01AA57BC4F73
:1033D00096E0FE01319601900D929A95E1F72093C7
:1033E00085030E94B0078091B603909185038917E9
:1033F00009F190E066E070E00E94F6218A579C4F48
:103400000E94F8178823B1F08091B60390E00196EE
:10341000877099278093B603E6CF0E94F30F10922E
:1034200085031092B60386E0EFE7F3E0DF011D921B
:103430008A95E9F767960FB6F894DEBF0FBECDBF49
:10344000DF91CF910895CF93DF9300D01F92CDB736
:10345000DEB720916903243041F520911001222329
:1034600021F123E029839B838A8382E08093E90012
:103470008FEF9091E800815095FD06C095ED9A95EB
:10348000F1F700008111F5CF8091E80085FF0DC0B4
:1034900050E040E063E070E0CE0101960E94220C13
:1034A0008091E8008E778093E8000F900F900F9046
:1034B000DF91CF910895CF93DF9300D01F92CDB7C6
:1034C000DEB720916903243081F520911001222379
:1034D00061F119821A821B8222E0298381389105C9
:1034E00020F0805891099B838A8382E08093E900D1
:1034F0008FEF9091E800815095FD06C095ED9A956B
:10350000F1F700008111F5CF8091E80085FF0DC033
:1035100050E040E063E070E0CE0101960E94220C92
:103520008091E8008E778093E8000F900F900F90C5
:10353000DF91CF91089520916903243049F522E06D
:103540002093E9002FEF3091E800215035FD06C0AF
:1035500035ED3A95F1F700002111F5CF2091E80003
:1035600025FF16C02091100150E040E063E070E0BC
:10357000222339F021E02093F10050E040E065E0A3
:1035800070E00E94220C8091E8008E778093E80022
:103590000895CF93DF9320916903243011F521E042
:1035A0002093E90021E8215021F03091E80035FF17
:1035B0001BC02091E80025FF14C0EC0150E040E062
:1035C00068E070E00E94220C8091E8008E77809382
:1035D000E80088E0FE01A6E5B3E001900D928A952F
:1035E000E1F7DF91CF910895EFE3F1E03197F1F743
:1035F00000C00000D8CFEF92FF921F93CF93DF93CC
:103600008CE5E82E81E0F82E1FEF0E94520DEC01B0
:103610001150CF3FDC0741F48FE99FE00197F1F7AC
:1036200000C000001111F1CF5C9A85ED8A95F1F789
:1036300000005C98DF93CF93FF92EF920E94DA052F
:103640000F900F900F900F90CB3FD105E9F2CE0174
:10365000DF91CF911F91FF90EF900895CF93C82FE6
:103660001F928F9385E591E09F938F930E94DA05D7
:103670005C9A8FE99FE00197F1F700C000000F907E
:103680000F900F900F908091C80085FFFCCFC093E2
:10369000CE008FE99FE00197F1F700C000005C9831
:1036A000CF910895EF92FF920F931F93CF93DF93E3
:1036B0000E94520D182FC82FD92FCF3FDC0709F0D9
:1036C00050C080913F03882309F444C004E711E00F
:1036D00023E6E22E21E0F22E8DE90E942E1B0E94AD
:1036E000FB1AEC01CF3FDC0791F18091500480FF81
:1036F0000AC0DF93CF931F930F930E94DA050F90B8
:103700000F900F900F90CA3FD10509F580913F03AC
:103710000E942E1B0E94FB1AEC01CF3FDC07E1F256
:103720008091500480FF10C0DF93CF9380913F03BE
:103730001F928F93FF92EF920E94DA050F900F90E5
:103740000F900F900F900F90CA3FD10529F610925D
:103750003F0380E0DF91CF911F910F91FF90EF9099
:1037600008959F931F9383E891E09F938F930E9406
:10377000DA05812F9E0193E0369527959A95E1F71A
:103780009C2F977061E070E0DB0102C0AA0FBB1FA5
:103790009A95E2F7E22FEF70F0E00F900F900F9004
:1037A0000F90E259FC4F408150E04A235B2317FF02
:1037B00018C0452B79F02F703327F901E259FC4FDF
:1037C000C770DD2701C0660FCA95EAF76095908142
:1037D000692360835C9A95ED9A95F1F700005C98F7
:1037E000B9CF452BB9F72F703327F901E259FC4FB8
:1037F000C770DD2701C0660FCA95EAF79081692B73
:10380000E8CF78941F920F920FB60F9211248F93E6
:103810009F93AF93BF9380914A0490914B04A091E2
:103820004C04B0914D040196A11DB11D80934A0432
:1038300090934B04A0934C04B0934D04BF91AF916F
:103840009F918F910F900FBE0F901F9018951F9210
:103850000F920FB60F9211248F939F93AF93BF9344
:1038600080913E04811113C080914A0490914B04D1
:10387000A0914C04B0914D044196A11DB11D8093BF
:103880004A0490934B04A0934C04B0934D04BF9111
:10389000AF919F918F910F900FBE0F901F90189531
:1038A0001F920F920FB60F9211242F933F934F93B5
:1038B0005F936F937F938F939F93AF93BF93EF9398
:1038C000FF938091E10082FF09C08091E20082FFB6
:1038D00005C08091E1008B7F8093E1008091E10041
:1038E00080FF1FC08091E20080FF1BC08091E2003A
:1038F0008E7F8093E2008091E20080618093E200FD
:103900008091D80080628093D80019BC85E08093B4
:1039100069038091550380935403109255030E94CC
:10392000F30F8091E10084FF2DC08091E20084FFBD
:1039300029C084E089BD86E089BD09B400FEFDCFC1
:103940008091D8008F7D8093D8008091E1008F7E98
:103950008093E1008091E2008F7E8093E20080916D
:10396000E20081608093E20080916003882309F483
:1039700040C084E0809369030E94F30F8091540358
:10398000809355038091E10083FF22C08091E20083
:1039900083FF1EC08091E100877F8093E10082E079
:1039A00080936903109260038091E1008E7F809381
:1039B000E1008091E2008E7F8093E2008091E2003E
:1039C00080618093E20042E060E080E00E94F208C3
:1039D000FF91EF91BF91AF919F918F917F916F91E7
:1039E0005F914F913F912F910F900FBE0F901F90BD
:1039F00018958091E30087FD02C081E0BBCF83E092
:103A0000B9CFCF93DF93CDB7DEB72C970FB6F8942D
:103A1000DEBF0FBECDBF84B7877F84BF0FB6F894DB
:103A2000A89580916000886180936000109260008A
:103A30000FBE80E890E00FB6F894809361009093F9
:103A400061000FBE89E69CE09093330180933201C0
:103A500086E091E090934204809341048AE492E0EE
:103A60000E9441050E941208809163008E7F80931E
:103A7000630081E0809353031092E2001092E10012
:103A80008091D8008F778093D8008091D80080688B
:103A90008093D8008091D8008F7D8093D80084E0F7
:103AA00089BD86E089BD09B400FEFDCF109269038F
:103AB0001092600310925F0310925E0342E060E098
:103AC00080E00E94F2088091E1008E7F8093E10007
:103AD0008091E20081608093E2008091E200886042
:103AE0008093E2008091E0008E7F8093E0007894E4
:103AF00082E084BD93E095BD9AEF97BD80936E0000
:103B00005B9A539A5C9A549A599A519A5C9A5B9828
:103B100020E52A95F1F75B9A83E38093CC0010921D
:103B2000CD008091C90080698093C9008091C9004F
:103B300088608093C9008091CA0080638093CA0026
:103B400052985A9A78943FEF49E688E131504040C4
:103B50008040E1F700C0000087ED91E09F938F93D4
:103B60000E94DA058FE90E942E1B0E94FB1A0F901B
:103B70000F908A3F910509F0DAC10E94FB1A803A42
:103B8000910509F0D4C10E94FB1A8038910509F013
:103B9000CEC181ED91E09F938F930E94DA050F9043
:103BA0000F9089EB91E09F938F930E94DA050F901D
:103BB0000F9019E9E12E11E0F12E0AE8C02E01E084
:103BC000D02E8CE90E942E1B0E94FB1A8C010F3F05
:103BD000100751F18091500480FF0AC01F930F938A
:103BE000FF92EF920E94DA050F900F900F900F90C6
:103BF0000A3F1105C9F480E70E942E1B0E94FB1AA0
:103C00008C010196F1F28091500480FF0AC01F934D
:103C10000F93DF92CF920E94DA050F900F900F90D2
:103C20000F900A3F110569F688EA91E09F938F9300
:103C30000E94DA050F900F9085E90E942E1B0E94CA
:103C4000FB1A8A3F910541F483E00E942E1B0E94DB
:103C5000FB1A8A3F910581F78EE793E0BEE6CB2EF3
:103C6000B3E0DB2EF60111926F018E179F07D1F79B
:103C70005C9880916903843009F05CC10E94510C0A
:103C8000882309F457C188E392E00E9441058AE243
:103C900092E00E944105F0E14F2EF2E05F2EAFE18D
:103CA0006A2EA2E07A2E80916903853009F445C11D
:103CB0000E94521B01E413E0EEE6AE2EE3E0BE2EBE
:103CC000312CF50121905F01F8019080921409F4E4
:103CD00068C08091500481FF40C083EF91E00E9452
:103CE00041052EE633E03C872B87F12CE12CEB8558
:103CF000FC852191FC87EB87229530E0C901880F74
:103D0000991F880F991F8C7C359527953595279598
:103D10002373822B90E028E131E03F932F939C01A5
:103D2000220F331F2A7A959587958575822B1F92CE
:103D30008F93FF92EF9288EE91E09F938F930E9472
:103D4000DA05FFEFEF1AFF0A0FB6F894DEBF0FBED9
:103D5000CDBF30E1E316F10451F6E12CFF24F394DA
:103D60009224892D8F21C1F0EE823F8291E0822D35
:103D70008F2109F490E098870E9492068160782F45
:103D80009A8789874E815F8168858A850E9492190A
:103D9000F80180818F258083E394FF0CF8E0EF1217
:103DA000E0CF33940F5F1F4F20E132128ACF8FEFA5
:103DB00089838A831B820E9492068160782F9D836B
:103DC0008C8349815A816B818D810E9492198091E7
:103DD0004304909144042FB7F89440914A045091C1
:103DE0004B0460914C0470914D042FBFFA01E81B05
:103DF000F90B209140048091160190E0211107C039
:103E00008091170190E06AE070E00E94F621E817C7
:103E1000F90780F08091460410914704009148040E
:103E2000F09049048111C1C0111181C101117FC1FC
:103E3000F1107DC10E94060890914003891709F492
:103E400041C00E94060880934003909150049570F1
:103E5000953051F41F928F937F926F920E94DA05F2
:103E60000F900F900F900F908091400390E780FD8E
:103E700091E790933F0381FF05C090913F039460C9
:103E800090933F039091500490FF0AC01F928F932C
:103E90005F924F920E94DA050F900F900F900F9053
:103EA0008091500480FF0EC080913F031F928F933A
:103EB00080E092E09F938F930E94DA050F900F901D
:103EC0000F900F902091E4003091E5008091510314
:103ED000909152032817390739F18091E4009091AD
:103EE000E50090935203809351030E94510C882364
:103EF000D9F0809169038430B9F48091E9008F7022
:103F00009091EC0090FFBFC090E8892B93E09093D4
:103F1000E9009091EB0090FF04C09091EE0097FDB6
:103F2000D0C08F708093E9000E942409BCCE8BEC36
:103F300091E031CE0E9424099CCE809169038430A7
:103F400021F110923E0488E190E020E40FB6F8944D
:103F5000A895809360000FBE2093600083B7817F97
:103F6000846083BF83B7816083BF7894889583B76B
:103F70008E7F83BF0FB6F894A8958091600088610A
:103F800080936000109260000FBE80915F038823D1
:103F900009F489CE0E94521BEEE6F3E08191811173
:103FA000B0C0CE16DF06D1F77ECE2F3F19F02F5FBF
:103FB00020934004181624F40E941E0680934604A1
:103FC0008091460487FF05C00E941E06819580935C
:103FD0004604111624F40E941E0680934704809123
:103FE000470487FF05C00E941E0681958093470401
:103FF00060914604662331F110914704112311F1B9
:10400000062E000C770B880B990B0E94F52023E3FA
:1040100033E343E35FE30E9459210E94BD20609394
:104020004604612F110F770B880B990B0E94F52026
:1040300023E333E343E35FE30E9459210E94BD2061
:1040400060934704101624F40E94E305809348040B
:104050008091480487FF05C00E94E3058195809305
:1040600048041F1424F40E94E305809349048091BE
:10407000490487FF05C00E94E305819580934904A8
:104080000E94F70ED7CE90E040CFE0910101F09171
:104090000201E90FF11D20819F5F309105019323FB
:1040A000909304012093F1009091E80095FD09C0E0
:1040B0009091E80090FF05C09091E8009E77909362
:1040C000E8009091040120910301291721F020912B
:1040D000E80025FDDACF9091F200992309F421CF71
:1040E0009091E80090FF1DCF9091E80095FD06C0EB
:1040F0009091E8009E779093E80013CF1092F10022
:10410000F3CF84E089BD86E089BD09B400FEFDCF10
:104110008091D8008F7D8093D8008091E0008260EC
:104120008093E0008091E00081FDFCCFBCCD2F3F6B
:1041300009F03DCF4ECF1F920F920FB60F92112470
:104140008F939F93EF93FF9380913D03E82FF0E0CF
:104150008F5F90913C03981739F09091CE00E45C0A
:10416000FD4F908380933D03FF91EF919F918F913D
:104170000F900FBE0F901F9018950E94C420689456
:10418000B1110C94532108950E94382188F09F5753
:1041900098F0B92F9927B751B0F0E1F0660F771F6B
:1041A000881F991F1AF0BA95C9F714C0B13091F061
:1041B0000E945221B1E008950C945221672F782F6C
:1041C0008827B85F39F0B93FCCF386957795679526
:1041D000B395D9F73EF490958095709561957F4F92
:1041E0008F4F9F4F0895E89409C097FB3EF4909538
:1041F0008095709561957F4F8F4F9F4F9923A9F0C0
:10420000F92F96E9BB279395F6958795779567954E
:10421000B795F111F8CFFAF4BB0F11F460FF1BC092
:104220006F5F7F4F8F4F9F4F16C0882311F096E925
:1042300011C0772321F09EE8872F762F05C06623D3
:1042400071F096E8862F70E060E02AF09A95660F8C
:10425000771F881FDAF7880F9695879597F9089545
:1042600057FD9058440F551F59F05F3F71F0479527
:10427000880F97FB991F61F09F3F79F0879508950C
:10428000121613061406551FF2CF4695F1DF08C02B
:10429000161617061806991FF1CF86957105610548
:1042A00008940895E894BB2766277727CB0197F9F0
:1042B00008950E946B210C94E5210E94D72138F0CB
:1042C0000E94DE2120F0952311F00C94CE210C9455
:1042D000D4210C9453210E94302178F39923C9F3FF
:1042E0005523B9F3950F50E0551FAA27EE27FF2756
:1042F000BB2700240894679520F4E20FF31FB41F36
:104300000A1E220F331F441FAA1F6695A9F777952F
:1043100030F4F30FB41F0A1E121E08F46395330F16
:10432000441FAA1F221F769599F7879520F4B40F92
:104330000A1E121E631F440FAA1F221F331F8695D9
:10434000A9F7862F712D602D11249F5750409AF0A8
:10435000F1F088234AF0EE0FFF1FBB1F661F771F87
:10436000881F91505040A9F79E3F510580F00C9452
:10437000CE210C9453215F3FE4F3983ED4F386950D
:1043800077956795B795F795E7959F5FC1F7FE2BF2
:10439000880F911D9695879597F9089597F99F67CE
:1043A00080E870E060E008959FEF80EC08950024BD
:1043B0000A941616170618060906089500240A948A
:1043C00012161306140605060895092E0394000C10
:1043D00011F4882352F0BB0F40F4BF2B11F460FF9F
:1043E00004C06F5F7F4F8F4F9F4F08950024552764
:1043F00004C0080E591F880F991F009729F0769561
:104400006795B8F37105B9F7802D952F089597FB3F
:10441000072E16F4009407D077FD09D00E942122C0
:1044200007FC05D03EF4909581959F4F08957095B7
:1044300061957F4F0895EE0FFF1F0590F491E02DD9
:104440000994AA1BBB1B51E107C0AA1FBB1FA617DB
:10445000B70710F0A61BB70B881F991F5A95A9F72D
:0E44600080959095BC01CD010895F894FFCF92
:10446E000534010000FF4E0CC91A9B1A5B1A231A61
:10447E0001012808140A321E00407F221501960001
:10448E00740075028E02A7020102030405060708D6
:02449E00090013
:10680000880000000000E2440400050006000700C4
:10681000080009000A000B000C000D000E000F001C
:1068200010001100120013001400150016001700CC
:10683000180019001A001B001C001D001E001F007C
:10684000200021002200230024002500260027002C
:10685000280029002A002B002C002D002E002F00DC
:1068600030003100000033003400000036003700F3
:10687000380082003A003B003C003D003E003F00F3
:106880004000410042004300440045004600000033
:10689000000049004A004B004C004D004E004F00E4
:1068A000500051005200000054005500560057009F
:1068B000000059005A005B005C005D005E005F0054
:1068C00060006100620063000000650085006700F1
:1068D000680069006A00000000000000000000007D
:1068E0000000000000000000890087008A008B0083
:1068F000E000E100E200E3000000E5000000E70046
:00000001FF
